******************************************************************************
                  TI ARM Linker PC v20.2.4                     
******************************************************************************
>> Linked Fri Mar 19 15:07:48 2021

OUTPUT FILE NAME:   <enet_adcsensor_client_lwip.out>
ENTRY POINT SYMBOL: "_c_int00_noargs"  address: 0000af81


MEMORY CONFIGURATION

         name            origin    length      used     unused   attr    fill
----------------------  --------  ---------  --------  --------  ----  --------
  FLASH                 00000000   00100000  0000bcfa  000f4306  R  X
  SRAM                  20000000   00040000  0001830d  00027cf3  RW X


SEGMENT ALLOCATION MAP

run origin  load origin   length   init length attrs members
----------  ----------- ---------- ----------- ----- -------
00000000    00000000    0000bd00   0000bd00    r-x
  00000000    00000000    00000200   00000200    r-- .intvecs
  00000200    00000200    0000b6e2   0000b6e2    r-x .text
  0000b8e4    0000b8e4    000003c0   000003c0    r-- .const
  0000bca8    0000bca8    00000058   00000058    r-- .cinit
20000000    20000000    0001830d   00000000    rw-
  20000000    20000000    00017a98   00000000    rw- .bss
  20017a98    20017a98    00000800   00000000    rw- .stack
  20018298    20018298    00000075   00000000    rw- .data


SECTION ALLOCATION MAP

 output                                  attributes/
section   page    origin      length       input sections
--------  ----  ----------  ----------   ----------------
.intvecs   0    00000000    00000200     
                  00000000    00000200     startup_ccs.obj (.intvecs)

.text      0    00000200    0000b6e2     
                  00000200    00000bc4     lwiplib.obj (.text:tcp_receive)
                  00000dc4    0000060c     lwiplib.obj (.text:tcp_process)
                  000013d0    00000580     lwiplib.obj (.text:tcp_input)
                  00001950    00000494     lwiplib.obj (.text:tcp_write)
                  00001de4    00000448     lwiplib.obj (.text:tcp_slowtmr)
                  0000222c    00000438     ustdlib.obj (.text:uvsnprintf)
                  00002664    000003f0     lwiplib.obj (.text:dhcp_parse_reply)
                  00002a54    0000030c     uartstdio.obj (.text:UARTvprintf)
                  00002d60    00000298     lwiplib.obj (.text:udp_input)
                  00002ff8    00000290     lwiplib.obj (.text:ip_input)
                  00003288    00000288     lwiplib.obj (.text:tivaif_receive)
                  00003510    00000280     enet_adcsensor_client_lwip.obj (.text:main)
                  00003790    0000026c     pinout.obj (.text:PinoutSet)
                  000039fc    00000244     lwiplib.obj (.text:tcp_output)
                  00003c40    0000023c     lwiplib.obj (.text:tcp_close_shutdown)
                  00003e7c    00000228     lwiplib.obj (.text:etharp_find_entry)
                  000040a4    0000020e     lwiplib.obj (.text:pbuf_alloc)
                  000042b2    00000206     lwiplib.obj (.text:ipaddr_aton)
                  000044b8    00000200     driverlib.lib : sysctl.obj (.text:SysCtlClockFreqSet)
                  000046b8    000001fc     lwiplib.obj (.text:dhcp_create_msg)
                  000048b4    000001e4     lwiplib.obj (.text:icmp_input)
                  00004a98    000001c4     lwiplib.obj (.text:etharp_query)
                  00004c5c    000001c0     lwiplib.obj (.text:etharp_arp_input)
                  00004e1c    000001b8     lwiplib.obj (.text:tivaif_transmit)
                  00004fd4    000001b6     rtsv7M4_T_le_v4SPD16_eabi.lib : fd_add_t2.asm.obj (.text)
                  0000518a    00000002     startup_ccs.obj (.text:FaultISR)
                  0000518c    000001b0     lwiplib.obj (.text:InitDMADescriptors)
                  0000533c    000001a8     lwiplib.obj (.text:etharp_output)
                  000054e4    000001a8     lwiplib.obj (.text:tcp_connect)
                  0000568c    0000019c     lwiplib.obj (.text:mem_trim)
                  00005828    00000188     lwiplib.obj (.text:mem_malloc)
                  000059b0    00000178     lwiplib.obj (.text:tcp_enqueue_flags)
                  00005b28    00000170     lwiplib.obj (.text:tcp_listen_input)
                  00005c98    0000016c     driverlib.lib : gpio.obj (.text:GPIOPadConfigSet)
                  00005e04    0000015c     lwiplib.obj (.text:autoip_tmr)
                  00005f60    0000014e     lwiplib.obj (.text:dhcp_bind)
                  000060ae    00000002     startup_ccs.obj (.text:IntDefaultHandler)
                  000060b0    00000138     lwiplib.obj (.text:dhcp_recv)
                  000061e8    00000136     rtsv7M4_T_le_v4SPD16_eabi.lib : fd_div_t2.asm.obj (.text)
                  0000631e    00000002     startup_ccs.obj (.text:NmiSR)
                  00006320    0000012c     lwiplib.obj (.text:tcp_output_segment)
                  0000644c    00000128     lwiplib.obj (.text:tcp_alloc)
                  00006574    0000011c     lwiplib.obj (.text:pbuf_copy)
                  00006690    00000118     lwiplib.obj (.text:udp_sendto_if)
                  000067a8    00000114     lwiplib.obj (.text:dhcp_select)
                  000068bc    00000108     lwiplib.obj (.text:dhcp_discover)
                  000069c4    00000104     lwiplib.obj (.text:etharp_raw)
                  00006ac8    00000104     lwiplib.obj (.text:memp_init)
                  00006bcc    00000104     lwiplib.obj (.text:tcp_parseopt)
                  00006cd0    000000fc     lwiplib.obj (.text:dhcp_start)
                  00006dcc    000000fc     lwiplib.obj (.text:etharp_update_arp_entry)
                  00006ec8    000000fc     rtsv7M4_T_le_v4SPD16_eabi.lib : fd_mul_t2.asm.obj (.text)
                  00006fc4    000000f8     lwiplib.obj (.text:ethernet_input)
                  000070bc    000000f0     lwiplib.obj (.text:lwIPInit)
                  000071ac    000000ec     lwiplib.obj (.text:ip_output_if)
                  00007298    000000e8     lwiplib.obj (.text:dhcp_release)
                  00007380    000000e8     lwiplib.obj (.text:pbuf_copy_partial)
                  00007468    000000e8     lwiplib.obj (.text:tcp_create_segment)
                  00007550    000000e4     lwiplib.obj (.text:lwIPServiceTimers)
                  00007634    000000dc     lwiplib.obj (.text:pbuf_header)
                  00007710    000000dc     lwiplib.obj (.text:tcp_bind)
                  000077ec    000000dc     lwiplib.obj (.text:tivaif_hwinit)
                  000078c8    000000d8     lwiplib.obj (.text:tcp_zero_window_probe)
                  000079a0    000000d4     lwiplib.obj (.text:sys_timeout)
                  00007a74    000000d0     lwiplib.obj (.text:dhcp_reboot)
                  00007b44    000000cc     enet_adcsensor_client_lwip.obj (.text:echoClientInit)
                  00007c10    000000c4     enet_adcsensor_client_lwip.obj (.text:TcpSendPacket)
                  00007cd4    000000c4     enet_adcsensor_client_lwip.obj (.text:connectCallback)
                  00007d98    000000c0     lwiplib.obj (.text:etharp_tmr)
                  00007e58    000000c0     lwiplib.obj (.text:netif_set_ipaddr)
                  00007f18    000000c0     lwiplib.obj (.text:udp_bind)
                  00007fd8    000000be     lwiplib.obj (.text:dhcp_timeout)
                  00008096    00000002     lwiplib.obj (.text:netif_init)
                  00008098    000000bc     lwiplib.obj (.text:dhcp_handle_ack)
                  00008154    000000bc     lwiplib.obj (.text:tcp_abandon)
                  00008210    000000bc     lwiplib.obj (.text:tcp_process_refused_data)
                  000082cc    000000b6     lwiplib.obj (.text:pbuf_realloc)
                  00008382    00000002     rtsv7M4_T_le_v4SPD16_eabi.lib : div0.asm.obj (.text)
                  00008384    000000b4     lwiplib.obj (.text:dhcp_rebind)
                  00008438    000000b4     lwiplib.obj (.text:raw_input)
                  000084ec    000000b4     lwiplib.obj (.text:tcp_oos_insert_segment)
                  000085a0    000000b2     lwiplib.obj (.text:dhcp_renew)
                  00008652    000000b2     lwiplib.obj (.text:lwip_standard_chksum)
                  00008704    000000b0     lwiplib.obj (.text:tcp_timewait_input)
                  000087b4    000000ac     lwiplib.obj (.text:autoip_arp_reply)
                  00008860    000000ac     lwiplib.obj (.text:dhcp_decline)
                  0000890c    000000ac     lwiplib.obj (.text:plug_holes)
                  000089b8    000000ac     lwiplib.obj (.text:tcp_output_alloc_header)
                  00008a64    000000a8     lwiplib.obj (.text:lwIPLinkDetect)
                  00008b0c    000000a8     lwiplib.obj (.text:memp_malloc)
                  00008bb4    000000a8     lwiplib.obj (.text:pbuf_free)
                  00008c5c    000000a8     lwiplib.obj (.text:tcp_write_checks)
                  00008d04    000000a8     lwiplib.obj (.text:tivaif_process_transmit)
                  00008dac    000000a6     lwiplib.obj (.text:tcp_pbuf_prealloc)
                  00008e52    00000002     lwiplib.obj (.text:stats_init)
                  00008e54    000000a0     lwiplib.obj (.text:icmp_send_response)
                  00008ef4    000000a0     lwiplib.obj (.text:inet_chksum_pbuf)
                  00008f94    000000a0     lwiplib.obj (.text:tcp_pcb_remove)
                  00009034    000000a0     lwiplib.obj (.text:tivaif_process_phy_interrupt)
                  000090d4    0000009c     enet_adcsensor_client_lwip.obj (.text:lwIPHostTimerHandler)
                  00009170    0000009c     rtsv7M4_T_le_v4SPD16_eabi.lib : memcpy_t2.asm.obj (.text)
                  0000920c    00000098     lwiplib.obj (.text:tcp_rst)
                  000092a4    00000094     lwiplib.obj (.text:autoip_start)
                  00009338    00000094     lwiplib.obj (.text:tcp_new_port)
                  000093cc    0000008e     lwiplib.obj (.text:tcp_rexmit_fast)
                  0000945a    00000002     lwiplib.obj (.text:tcp_init)
                  0000945c    0000008c     lwiplib.obj (.text:lwIPEthernetIntHandler)
                  000094e8    0000008c     lwiplib.obj (.text:udp_connect)
                  00009574    00000088     lwiplib.obj (.text:mem_free)
                  000095fc    00000088     lwiplib.obj (.text:tcp_fasttmr)
                  00009684    00000084     lwiplib.obj (.text:ip_route)
                  00009708    00000084     lwiplib.obj (.text:lwIPPrivateInit)
                  0000978c    00000084     lwiplib.obj (.text:netif_add)
                  00009810    00000084     lwiplib.obj (.text:tcp_kill_prio)
                  00009894    00000080     lwiplib.obj (.text:etharp_output_to_arp_index)
                  00009914    0000007c     lwiplib.obj (.text:autoip_start_probing)
                  00009990    0000007c     lwiplib.obj (.text:mem_init)
                  00009a0c    0000007c     lwiplib.obj (.text:tcp_rexmit)
                  00009a88    0000007a     driverlib.lib : adc.obj (.text:ADCSequenceStepConfigure)
                  00009b02    0000007a     rtsv7M4_T_le_v4SPD16_eabi.lib : memset_t2.asm.obj (.text)
                  00009b7c    00000078     driverlib.lib : emac.obj (.text:EMACInit)
                  00009bf4    00000076     lwiplib.obj (.text:tcp_update_rcv_ann_wnd)
                  00009c6a    00000002     lwiplib.obj (.text:udp_init)
                  00009c6c    00000074     uartstdio.obj (.text:UARTStdioConfig)
                  00009ce0    00000074     lwiplib.obj (.text:autoip_create_addr)
                  00009d54    00000072     lwiplib.obj (.text:dhcp_option_long)
                  00009dc6    0000006c     lwiplib.obj (.text:ip4_addr_isbroadcast)
                  00009e32    00000002     --HOLE-- [fill = 0]
                  00009e34    0000006c     lwiplib.obj (.text:udp_new_port)
                  00009ea0    0000006a     lwiplib.obj (.text:tcp_pcb_purge)
                  00009f0a    00000002     --HOLE-- [fill = 0]
                  00009f0c    00000068     driverlib.lib : interrupt.obj (.text:IntEnable)
                  00009f74    00000068     rtsv7M4_T_le_v4SPD16_eabi.lib : copy_decompress_lzss.c.obj (.text:decompress:lzss:__TI_decompress_lzss)
                  00009fdc    00000068     lwiplib.obj (.text:tivaif_check_pbuf)
                  0000a044    00000066     lwiplib.obj (.text:tcp_send_empty_ack)
                  0000a0aa    00000002     --HOLE-- [fill = 0]
                  0000a0ac    00000064     uartstdio.obj (.text:UARTwrite)
                  0000a110    00000064     lwiplib.obj (.text:etharp_cleanup_netif)
                  0000a174    00000062     lwiplib.obj (.text:dhcp_network_changed)
                  0000a1d6    0000005c     lwiplib.obj (.text:tcp_send_fin)
                  0000a232    00000002     --HOLE-- [fill = 0]
                  0000a234    00000058     driverlib.lib : emac.obj (.text:EMACPHYConfigSet)
                  0000a28c    00000058     lwiplib.obj (.text:tcp_keepalive)
                  0000a2e4    00000058     lwiplib.obj (.text:tivaif_interrupt)
                  0000a33c    00000058     lwiplib.obj (.text:udp_remove)
                  0000a394    00000058     ustdlib.obj (.text:ustrncpy)
                  0000a3ec    00000054     lwiplib.obj (.text:dhcp_fine_tmr)
                  0000a440    00000054     lwiplib.obj (.text:memp_free)
                  0000a494    00000054     lwiplib.obj (.text:netif_set_link_up)
                  0000a4e8    00000054     lwiplib.obj (.text:tcp_kill_timewait)
                  0000a53c    00000052     lwiplib.obj (.text:dhcp_option_trailer)
                  0000a58e    00000052     lwiplib.obj (.text:dhcp_stop)
                  0000a5e0    00000050     driverlib.lib : sysctl.obj (.text:SysCtlPeripheralReset)
                  0000a630    00000050     lwiplib.obj (.text:dhcp_coarse_tmr)
                  0000a680    00000050     lwiplib.obj (.text:sys_timeouts_init)
                  0000a6d0    00000050     lwiplib.obj (.text:tcp_rexmit_rto)
                  0000a720    0000004e     driverlib.lib : adc.obj (.text:ADCSequenceConfigure)
                  0000a76e    00000002     --HOLE-- [fill = 0]
                  0000a770    0000004c     lwiplib.obj (.text:ip_output)
                  0000a7bc    00000048     driverlib.lib : sysctl.obj (.text:_SysCtlFrequencyGet)
                  0000a804    00000048     lwiplib.obj (.text:dhcp_check)
                  0000a84c    00000048     lwiplib.obj (.text:etharp_free_entry)
                  0000a894    00000048     lwiplib.obj (.text:tcp_recved)
                  0000a8dc    00000046     lwiplib.obj (.text:pbuf_cat)
                  0000a922    00000002     --HOLE-- [fill = 0]
                  0000a924    00000044     enet_adcsensor_client_lwip.obj (.text:DisplayIPAddress)
                  0000a968    00000044     rtsv7M4_T_le_v4SPD16_eabi.lib : autoinit.c.obj (.text:__TI_auto_init_nobinit_nopinit:__TI_auto_init_nobinit_nopinit)
                  0000a9ac    00000044     lwiplib.obj (.text:dhcp_option_short)
                  0000a9f0    00000044     lwiplib.obj (.text:etharp_send_ip)
                  0000aa34    00000044     rtsv7M4_T_le_v4SPD16_eabi.lib : fd_tou_t2.asm.obj (.text)
                  0000aa78    00000044     lwiplib.obj (.text:tcp_eff_send_mss)
                  0000aabc    00000044     lwiplib.obj (.text:tivaif_init)
                  0000ab00    00000040     rtsv7M4_T_le_v4SPD16_eabi.lib : u_divt2.asm.obj (.text)
                  0000ab40    0000003e     lwiplib.obj (.text:dhcp_option)
                  0000ab7e    00000002     --HOLE-- [fill = 0]
                  0000ab80    0000003c     enet_adcsensor_client_lwip.obj (.text:adcConfigure)
                  0000abbc    0000003c     lwiplib.obj (.text:autoip_arp_probe)
                  0000abf8    0000003c     lwiplib.obj (.text:autoip_bind)
                  0000ac34    0000003c     lwiplib.obj (.text:dhcp_handle_nak)
                  0000ac70    0000003c     lwiplib.obj (.text:netif_set_up)
                  0000acac    0000003a     driverlib.lib : emac.obj (.text:EMACIntEnable)
                  0000ace6    0000003a     lwiplib.obj (.text:autoip_handle_arp_conflict)
                  0000ad20    0000003a     lwiplib.obj (.text:tcp_recv_null)
                  0000ad5a    00000002     --HOLE-- [fill = 0]
                  0000ad5c    00000038     driverlib.lib : emac.obj (.text:EMACConfigSet)
                  0000ad94    00000038                   : sysctl.obj (.text:SysCtlPeripheralReady)
                  0000adcc    00000038     lwiplib.obj (.text:autoip_arp_announce)
                  0000ae04    00000038     lwiplib.obj (.text:dhcp_handle_offer)
                  0000ae3c    00000038     lwiplib.obj (.text:etharp_request)
                  0000ae74    00000038     lwiplib.obj (.text:tcp_timer_needed)
                  0000aeac    00000038     lwiplib.obj (.text:tcpip_tcp_timer)
                  0000aee4    00000034     driverlib.lib : emac.obj (.text:EMACConfigGet)
                  0000af18    00000034                   : emac.obj (.text:EMACIntClear)
                  0000af4c    00000034                   : sysctl.obj (.text:SysCtlPeripheralEnable)
                  0000af80    00000034     rtsv7M4_T_le_v4SPD16_eabi.lib : boot_cortex_m.c.obj (.text:_c_int00_noargs:_c_int00_noargs)
                  0000afb4    00000032     ustdlib.obj (.text:usprintf)
                  0000afe6    00000030     lwiplib.obj (.text:dhcp_arp_reply)
                  0000b016    0000002e     driverlib.lib : adc.obj (.text:ADCIntStatus)
                  0000b044    0000002e     lwiplib.obj (.text:dhcp_set_state)
                  0000b072    0000002e     lwiplib.obj (.text:netif_set_down)
                  0000b0a0    0000002e     lwiplib.obj (.text:pbuf_clen)
                  0000b0ce    0000002c     driverlib.lib : emac.obj (.text:EMACIntStatus)
                  0000b0fa    0000002c                   : gpio.obj (.text:GPIODirModeSet)
                  0000b126    00000002     --HOLE-- [fill = 0]
                  0000b128    0000002c     enet_adcsensor_client_lwip.obj (.text:SysTickIntHandler)
                  0000b154    0000002c     lwiplib.obj (.text:lwip_htonl)
                  0000b180    0000002a     lwiplib.obj (.text:dhcp_t1_timeout)
                  0000b1aa    0000002a     lwiplib.obj (.text:dhcp_t2_timeout)
                  0000b1d4    0000002a     lwiplib.obj (.text:netif_set_addr)
                  0000b1fe    0000002a     lwiplib.obj (.text:tcp_seg_copy)
                  0000b228    00000028     lwiplib.obj (.text:lwIPTimer)
                  0000b250    00000026     driverlib.lib : emac.obj (.text:EMACPHYRead)
                  0000b276    00000026                   : emac.obj (.text:EMACPHYWrite)
                  0000b29c    00000024                   : interrupt.obj (.text:IntPrioritySet)
                  0000b2c0    00000024     uartstdio.obj (.text:UARTprintf)
                  0000b2e4    00000024     lwiplib.obj (.text:dhcp_delete_msg)
                  0000b308    00000024     lwiplib.obj (.text:dhcp_option_byte)
                  0000b32c    00000024     lwiplib.obj (.text:lwip_htons)
                  0000b350    00000024     rtsv7M4_T_le_v4SPD16_eabi.lib : memcmp.c.obj (.text:memcmp)
                  0000b374    00000022     lwiplib.obj (.text:netif_set_link_down)
                  0000b396    00000022     lwiplib.obj (.text:pbuf_ref)
                  0000b3b8    00000022     lwiplib.obj (.text:udp_new)
                  0000b3da    00000002     --HOLE-- [fill = 0]
                  0000b3dc    00000020     driverlib.lib : sysctl.obj (.text:_SysCtlMemTimingGet)
                  0000b3fc    00000020     lwiplib.obj (.text:autoip_network_changed)
                  0000b41c    00000020     lwiplib.obj (.text:lwip_init)
                  0000b43c    00000020     lwiplib.obj (.text:pbuf_pool_is_empty)
                  0000b45c    00000020     rtsv7M4_T_le_v4SPD16_eabi.lib : u_tofd_t2.asm.obj (.text)
                  0000b47c    00000020     lwiplib.obj (.text:tcp_close)
                  0000b49c    00000020     lwiplib.obj (.text:tcp_seg_free)
                  0000b4bc    00000020     lwiplib.obj (.text:tcp_segs_free)
                  0000b4dc    00000020     lwiplib.obj (.text:tcp_tmr)
                  0000b4fc    0000001e     driverlib.lib : adc.obj (.text:ADCSequenceDataGet)
                  0000b51a    0000001e                   : emac.obj (.text:EMACAddrGet)
                  0000b538    0000001c     lwiplib.obj (.text:arp_timer)
                  0000b554    0000001c     lwiplib.obj (.text:dhcp_timer_coarse)
                  0000b570    0000001c     lwiplib.obj (.text:dhcp_timer_fine)
                  0000b58c    0000001c     lwiplib.obj (.text:lwIPLocalIPAddrGet)
                  0000b5a8    0000001c     lwiplib.obj (.text:netif_set_gw)
                  0000b5c4    0000001c     lwiplib.obj (.text:netif_set_netmask)
                  0000b5e0    0000001c     lwiplib.obj (.text:sys_arch_unprotect)
                  0000b5fc    0000001c     lwiplib.obj (.text:tcp_next_iss)
                  0000b618    0000001a     driverlib.lib : gpio.obj (.text:GPIOPinTypeGPIOOutput)
                  0000b632    0000001a     lwiplib.obj (.text:udp_recv)
                  0000b64c    00000018     driverlib.lib : adc.obj (.text:ADCProcessorTrigger)
                  0000b664    00000018     lwiplib.obj (.text:autoip_timer)
                  0000b67c    00000018     lwiplib.obj (.text:inet_chksum)
                  0000b694    00000018     lwiplib.obj (.text:ipaddr_addr)
                  0000b6ac    00000016     driverlib.lib : emac.obj (.text:EMACReset)
                  0000b6c2    00000016                   : emac.obj (.text:EMACRxEnable)
                  0000b6d8    00000016                   : emac.obj (.text:EMACTxEnable)
                  0000b6ee    00000016                   : gpio.obj (.text:GPIOPinTypeEthernetLED)
                  0000b704    00000016     lwiplib.obj (.text:autoip_restart)
                  0000b71a    00000016     lwiplib.obj (.text:autoip_stop)
                  0000b730    00000016     lwiplib.obj (.text:icmp_dest_unreach)
                  0000b746    00000016     lwiplib.obj (.text:pbuf_chain)
                  0000b75c    00000014     driverlib.lib : flash.obj (.text:FlashUserGet)
                  0000b770    00000014                   : systick.obj (.text:SysTickEnable)
                  0000b784    00000014                   : systick.obj (.text:SysTickIntEnable)
                  0000b798    00000014     lwiplib.obj (.text:netif_set_default)
                  0000b7ac    00000014     rtsv7M4_T_le_v4SPD16_eabi.lib : strlen.c.obj (.text:strlen)
                  0000b7c0    00000012     lwiplib.obj (.text:tcp_sent)
                  0000b7d2    00000002     --HOLE-- [fill = 0]
                  0000b7d4    00000010     driverlib.lib : emac.obj (.text:EMACFrameFilterSet)
                  0000b7e4    00000010                   : interrupt.obj (.text:IntMasterEnable)
                  0000b7f4    00000010                   : systick.obj (.text:SysTickPeriodSet)
                  0000b804    00000010     lwiplib.obj (.text:lwip_ntohs)
                  0000b814    00000010     lwiplib.obj (.text:sys_arch_protect)
                  0000b824    0000000e     driverlib.lib : adc.obj (.text:ADCSequenceEnable)
                  0000b832    0000000e     rtsv7M4_T_le_v4SPD16_eabi.lib : copy_decompress_none.c.obj (.text:decompress:none:__TI_decompress_none)
                  0000b840    0000000e     lwiplib.obj (.text:tcp_abort)
                  0000b84e    0000000c     driverlib.lib : cpu.obj (.text:CPUcpsie)
                  0000b85a    00000002     --HOLE-- [fill = 0]
                  0000b85c    0000000c                   : sysctl.obj (.text:SysCtlMOSCConfigSet)
                  0000b868    0000000c     rtsv7M4_T_le_v4SPD16_eabi.lib : copy_zero_init.c.obj (.text:decompress:ZI:__TI_zero_init)
                  0000b874    0000000c     lwiplib.obj (.text:lwip_ntohl)
                  0000b880    0000000c     lwiplib.obj (.text:sys_now)
                  0000b88c    0000000a     driverlib.lib : adc.obj (.text:ADCIntClear)
                  0000b896    0000000a     lwiplib.obj (.text:tcp_new)
                  0000b8a0    00000008     driverlib.lib : emac.obj (.text:EMACPowerManagementStatusGet)
                  0000b8a8    00000008                   : emac.obj (.text:EMACTxDMAPollDemand)
                  0000b8b0    00000006                   : emac.obj (.text:EMACRxDMADescriptorListSet)
                  0000b8b6    00000006                   : emac.obj (.text:EMACTimestampIntStatus)
                  0000b8bc    00000006                   : emac.obj (.text:EMACTxDMADescriptorListSet)
                  0000b8c2    00000006                   : gpio.obj (.text:GPIOPinRead)
                  0000b8c8    00000006                   : gpio.obj (.text:GPIOPinWrite)
                  0000b8ce    00000006     startup_ccs.obj (.text:ResetISR)
                  0000b8d4    00000006     driverlib.lib : sysctl.obj (.text:SysCtlDelay)
                  0000b8da    00000004     rtsv7M4_T_le_v4SPD16_eabi.lib : pre_init.c.obj (.text:_system_pre_init)
                  0000b8de    00000004                                   : exit.c.obj (.text:abort:abort)

.const     0    0000b8e4    000003c0     
                  0000b8e4    000001b0     driverlib.lib : sysctl.obj (.const:g_pppui32XTALtoVCO)
                  0000ba94    0000009c                   : interrupt.obj (.const:g_pui32Regs)
                  0000bb30    0000006c                   : sysctl.obj (.const:g_pui32Xtals)
                  0000bb9c    00000030                   : sysctl.obj (.const:g_sXTALtoMEMTIM)
                  0000bbcc    00000018                   : emac.obj (.const:g_pi16MIIClockDiv)
                  0000bbe4    00000014                   : interrupt.obj (.const:g_pui32EnRegs)
                  0000bbf8    00000012     uartstdio.obj (.const:.string)
                  0000bc0a    00000002     --HOLE-- [fill = 0]
                  0000bc0c    00000012     ustdlib.obj (.const:.string)
                  0000bc1e    00000010     lwiplib.obj (.const:memp_num)
                  0000bc2e    00000010     lwiplib.obj (.const:memp_sizes)
                  0000bc3e    00000002     --HOLE-- [fill = 0]
                  0000bc40    00000010     lwiplib.obj (.const:tcp_pcb_lists)
                  0000bc50    0000000d     lwiplib.obj (.const:.string:tcp_backoff)
                  0000bc5d    00000003     --HOLE-- [fill = 0]
                  0000bc60    0000000c     uartstdio.obj (.const:g_ui32UARTBase)
                  0000bc6c    0000000c     uartstdio.obj (.const:g_ui32UARTPeriph)
                  0000bc78    00000008     driverlib.lib : sysctl.obj (.const:g_pui32VCOFrequencies)
                  0000bc80    00000007     lwiplib.obj (.const:.string:tcp_persist_backoff)
                  0000bc87    00000006     lwiplib.obj (.const:ethbroadcast)
                  0000bc8d    00000006     lwiplib.obj (.const:ethzero)
                  0000bc93    00000001     --HOLE-- [fill = 0]
                  0000bc94    00000004     lwiplib.obj (.const:ip_addr_any)
                  0000bc98    00000004     lwiplib.obj (.const:ip_addr_broadcast)
                  0000bc9c    00000004     uartstdio.obj (.const)
                  0000bca0    00000004     ustdlib.obj (.const)

.cinit     0    0000bca8    00000058     
                  0000bca8    00000033     (.cinit..data.load) [load image, compression = lzss]
                  0000bcdb    00000001     --HOLE-- [fill = 0]
                  0000bcdc    0000000c     (__TI_handler_table)
                  0000bce8    00000008     (.cinit..bss.load) [load image, compression = zero_init]
                  0000bcf0    00000010     (__TI_cinit_table)

.init_array 
*          0    00000000    00000000     UNINITIALIZED

.bss       0    20000000    00017a98     UNINITIALIZED
                  20000000    0001001c     (.common:ram_heap)
                  2001001c    000072d4     lwiplib.obj (.bss:memp_memory)
                  200172f0    00000360     (.common:g_pTxDescriptors)
                  20017650    00000120     (.common:g_pRxDescriptors)
                  20017770    00000120     (.common:lwip_stats)
                  20017890    000000c8     lwiplib.obj (.bss:arp_table)
                  20017958    00000050     lwiplib.obj (.bss)
                  200179a8    00000038     lwiplib.obj (.bss:g_sNetIF)
                  200179e0    00000028     (.common:dhcp_rx_options_val)
                  20017a08    00000020     lwiplib.obj (.bss:memp_tab)
                  20017a28    00000010     lwiplib.obj (.bss:inseg)
                  20017a38    0000000c     (.common:dhcp_rx_options_given)
                  20017a44    00000004     enet_adcsensor_client_lwip.obj (.bss)
                  20017a48    00000004     (.common:current_header)
                  20017a4c    00000004     (.common:current_iphdr_dest)
                  20017a50    00000004     (.common:current_iphdr_src)
                  20017a54    00000004     (.common:current_netif)
                  20017a58    00000004     (.common:g_pfnTimerHandler)
                  20017a5c    00000004     (.common:g_ui32AbnormalInts)
                  20017a60    00000004     (.common:g_ui32IPAddress)
                  20017a64    00000004     (.common:g_ui32NormalInts)
                  20017a68    00000004     (.common:g_ui32SysClock)
                  20017a6c    00000004     (.common:netif_default)
                  20017a70    00000004     (.common:netif_list)
                  20017a74    00000004     (.common:tcp_active_pcbs)
                  20017a78    00000004     (.common:tcp_bound_pcbs)
                  20017a7c    00000004     (.common:tcp_input_pcb)
                  20017a80    00000004     (.common:tcp_listen_pcbs)
                  20017a84    00000004     (.common:tcp_ticks)
                  20017a88    00000004     (.common:tcp_tmp_pcb)
                  20017a8c    00000004     (.common:tcp_tw_pcbs)
                  20017a90    00000004     (.common:udp_pcbs)
                  20017a94    00000001     (.common:err)
                  20017a95    00000001     (.common:g_bLED)
                  20017a96    00000001     (.common:pbuf_free_ooseq_pending)
                  20017a97    00000001     (.common:tcp_active_pcbs_changed)

.data      0    20018298    00000075     UNINITIALIZED
                  20018298    00000038     lwiplib.obj (.data)
                  200182d0    00000010     lwiplib.obj (.data:g_RxDescList)
                  200182e0    00000010     lwiplib.obj (.data:g_TxDescList)
                  200182f0    0000000c     enet_adcsensor_client_lwip.obj (.data)
                  200182fc    0000000c     lwiplib.obj (.data:g_StellarisIFData)
                  20018308    00000005     uartstdio.obj (.data)

.stack     0    20017a98    00000800     UNINITIALIZED
                  20017a98    00000004     rtsv7M4_T_le_v4SPD16_eabi.lib : boot_cortex_m.c.obj (.stack)
                  20017a9c    000007fc     --HOLE--

__llvm_prf_cnts 
*          0    20000000    00000000     UNINITIALIZED

MODULE SUMMARY

       Module                           code    ro data   rw data
       ------                           ----    -------   -------
    .\
       enet_adcsensor_client_lwip.obj   1564    0         26     
       startup_ccs.obj                  12      512       0      
    +--+--------------------------------+-------+---------+---------+
       Total:                           1576    512       26     
                                                                 
    .\drivers\
       pinout.obj                       620     0         0      
    +--+--------------------------------+-------+---------+---------+
       Total:                           620     0         0      
                                                                 
    .\utils\
       lwiplib.obj                      38040   88        97006  
       ustdlib.obj                      1218    22        0      
       uartstdio.obj                    1032    46        5      
    +--+--------------------------------+-------+---------+---------+
       Total:                           40290   156       97011  
                                                                 
    C:/ti/TivaWare_C_Series-2.2.0.295/driverlib/ccs/Debug/driverlib.lib
       sysctl.obj                       822     596       0      
       emac.obj                         692     24        0      
       gpio.obj                         468     0         0      
       interrupt.obj                    156     176       0      
       adc.obj                          324     0         0      
       systick.obj                      56      0         0      
       flash.obj                        20      0         0      
       cpu.obj                          12      0         0      
    +--+--------------------------------+-------+---------+---------+
       Total:                           2550    796       0      
                                                                 
    C:\ti\ccs1011\ccs\tools\compiler\ti-cgt-arm_20.2.4.LTS\lib\rtsv7M4_T_le_v4SPD16_eabi.lib
       fd_add_t2.asm.obj                438     0         0      
       fd_div_t2.asm.obj                310     0         0      
       fd_mul_t2.asm.obj                252     0         0      
       memcpy_t2.asm.obj                156     0         0      
       memset_t2.asm.obj                122     0         0      
       copy_decompress_lzss.c.obj       104     0         0      
       autoinit.c.obj                   68      0         0      
       fd_tou_t2.asm.obj                68      0         0      
       u_divt2.asm.obj                  64      0         0      
       boot_cortex_m.c.obj              52      0         0      
       memcmp.c.obj                     36      0         0      
       u_tofd_t2.asm.obj                32      0         0      
       strlen.c.obj                     20      0         0      
       copy_decompress_none.c.obj       14      0         0      
       copy_zero_init.c.obj             12      0         0      
       exit.c.obj                       4       0         0      
       pre_init.c.obj                   4       0         0      
       div0.asm.obj                     2       0         0      
    +--+--------------------------------+-------+---------+---------+
       Total:                           1758    0         0      
                                                                 
       Stack:                           0       0         2048   
       Linker Generated:                0       87        0      
    +--+--------------------------------+-------+---------+---------+
       Grand Total:                     46794   1551      99085  


LINKER GENERATED COPY TABLES

__TI_cinit_table @ 0000bcf0 records: 2, size/record: 8, table size: 16
	.data: load addr=0000bca8, load size=00000033 bytes, run addr=20018298, run size=00000075 bytes, compression=lzss
	.bss: load addr=0000bce8, load size=00000008 bytes, run addr=20000000, run size=00017a98 bytes, compression=zero_init


LINKER GENERATED HANDLER TABLE

__TI_handler_table @ 0000bcdc records: 3, size/record: 4, table size: 12
	index: 0, handler: __TI_decompress_lzss
	index: 1, handler: __TI_decompress_none
	index: 2, handler: __TI_zero_init


GLOBAL SYMBOLS: SORTED ALPHABETICALLY BY Name 

address   name                          
-------   ----                          
0000b88d  ADCIntClear                   
0000b017  ADCIntStatus                  
0000b64d  ADCProcessorTrigger           
0000a721  ADCSequenceConfigure          
0000b4fd  ADCSequenceDataGet            
0000b825  ADCSequenceEnable             
00009a89  ADCSequenceStepConfigure      
0000b8df  C$$EXIT                       
0000b84f  CPUcpsie                      
0000a925  DisplayIPAddress              
0000b51b  EMACAddrGet                   
0000aee5  EMACConfigGet                 
0000ad5d  EMACConfigSet                 
0000b7d5  EMACFrameFilterSet            
00009b7d  EMACInit                      
0000af19  EMACIntClear                  
0000acad  EMACIntEnable                 
0000b0cf  EMACIntStatus                 
0000a235  EMACPHYConfigSet              
0000b251  EMACPHYRead                   
0000b277  EMACPHYWrite                  
0000b8a1  EMACPowerManagementStatusGet  
0000b6ad  EMACReset                     
0000b8b1  EMACRxDMADescriptorListSet    
0000b6c3  EMACRxEnable                  
0000b8b7  EMACTimestampIntStatus        
0000b8bd  EMACTxDMADescriptorListSet    
0000b8a9  EMACTxDMAPollDemand           
0000b6d9  EMACTxEnable                  
0000b75d  FlashUserGet                  
0000b0fb  GPIODirModeSet                
00005c99  GPIOPadConfigSet              
0000b8c3  GPIOPinRead                   
0000b6ef  GPIOPinTypeEthernetLED        
0000b619  GPIOPinTypeGPIOOutput         
0000b8c9  GPIOPinWrite                  
0000518d  InitDMADescriptors            
00009f0d  IntEnable                     
0000b7e5  IntMasterEnable               
0000b29d  IntPrioritySet                
00003791  PinoutSet                     
0000b8cf  ResetISR                      
000044b9  SysCtlClockFreqSet            
0000b8d5  SysCtlDelay                   
0000b85d  SysCtlMOSCConfigSet           
0000af4d  SysCtlPeripheralEnable        
0000ad95  SysCtlPeripheralReady         
0000a5e1  SysCtlPeripheralReset         
0000b771  SysTickEnable                 
0000b785  SysTickIntEnable              
0000b129  SysTickIntHandler             
0000b7f5  SysTickPeriodSet              
00007c11  TcpSendPacket                 
00009c6d  UARTStdioConfig               
0000b2c1  UARTprintf                    
00002a55  UARTvprintf                   
0000a0ad  UARTwrite                     
20018298  __STACK_END                   
00000800  __STACK_SIZE                  
20018298  __STACK_TOP                   
0000bcf0  __TI_CINIT_Base               
0000bd00  __TI_CINIT_Limit              
0000bcdc  __TI_Handler_Table_Base       
0000bce8  __TI_Handler_Table_Limit      
0000a969  __TI_auto_init_nobinit_nopinit
00009f75  __TI_decompress_lzss          
0000b833  __TI_decompress_none          
ffffffff  __TI_pprof_out_hndl           
ffffffff  __TI_prof_data_size           
ffffffff  __TI_prof_data_start          
00000000  __TI_static_base__            
0000b869  __TI_zero_init                
0000aa35  __aeabi_d2uiz                 
00004fdf  __aeabi_dadd                  
000061e9  __aeabi_ddiv                  
00006ec9  __aeabi_dmul                  
00004fd5  __aeabi_dsub                  
00008383  __aeabi_idiv0                 
00008383  __aeabi_ldiv0                 
00009b03  __aeabi_memclr                
00009b03  __aeabi_memclr4               
00009b03  __aeabi_memclr8               
00009171  __aeabi_memcpy                
00009171  __aeabi_memcpy4               
00009171  __aeabi_memcpy8               
00009b05  __aeabi_memset                
00009b05  __aeabi_memset4               
00009b05  __aeabi_memset8               
0000b45d  __aeabi_ui2d                  
0000ab01  __aeabi_uidiv                 
0000ab01  __aeabi_uidivmod              
ffffffff  __binit__                     
ffffffff  __c_args__                    
UNDEFED   __mpu_init                    
20017a98  __stack                       
20000000  __start___llvm_prf_cnts       
20000000  __stop___llvm_prf_cnts        
0000af81  _c_int00_noargs               
UNDEFED   _system_post_cinit            
0000b8db  _system_pre_init              
0000b8df  abort                         
0000ab81  adcConfigure                  
000087b5  autoip_arp_reply              
0000b3fd  autoip_network_changed        
000092a5  autoip_start                  
0000b71b  autoip_stop                   
00005e05  autoip_tmr                    
ffffffff  binit                         
00007cd5  connectCallback               
20017a48  current_header                
20017a4c  current_iphdr_dest            
20017a50  current_iphdr_src             
20017a54  current_netif                 
0000afe7  dhcp_arp_reply                
0000a631  dhcp_coarse_tmr               
0000a3ed  dhcp_fine_tmr                 
0000a175  dhcp_network_changed          
00007299  dhcp_release                  
000085a1  dhcp_renew                    
20017a38  dhcp_rx_options_given         
200179e0  dhcp_rx_options_val           
00006cd1  dhcp_start                    
0000a58f  dhcp_stop                     
00007b45  echoClientInit                
20017a94  err                           
0000a111  etharp_cleanup_netif          
0000533d  etharp_output                 
00004a99  etharp_query                  
000069c5  etharp_raw                    
0000ae3d  etharp_request                
00007d99  etharp_tmr                    
0000bc87  ethbroadcast                  
00006fc5  ethernet_input                
0000bc8d  ethzero                       
200182d0  g_RxDescList                  
200182e0  g_TxDescList                  
200182f4  g_bIPAddrValid                
20017a95  g_bLED                        
200182f5  g_bconnect                    
20017650  g_pRxDescriptors              
200172f0  g_pTxDescriptors              
20017a58  g_pfnTimerHandler             
00000000  g_pfnVectors                  
20017a5c  g_ui32AbnormalInts            
20017a60  g_ui32IPAddress               
2001829c  g_ui32LocalTimer              
20017a64  g_ui32NormalInts              
20017a68  g_ui32SysClock                
200182f8  g_ui32sysTick                 
200182f0  g_ui32tcpPollTick             
0000b731  icmp_dest_unreach             
000048b5  icmp_input                    
0000b67d  inet_chksum                   
00008ef5  inet_chksum_pbuf              
00009dc7  ip4_addr_isbroadcast          
0000bc94  ip_addr_any                   
0000bc98  ip_addr_broadcast             
00002ff9  ip_input                      
0000a771  ip_output                     
000071ad  ip_output_if                  
00009685  ip_route                      
0000b695  ipaddr_addr                   
000042b3  ipaddr_aton                   
0000945d  lwIPEthernetIntHandler        
000090d5  lwIPHostTimerHandler          
000070bd  lwIPInit                      
0000b58d  lwIPLocalIPAddrGet            
0000b229  lwIPTimer                     
0000b155  lwip_htonl                    
0000b32d  lwip_htons                    
0000b41d  lwip_init                     
0000b875  lwip_ntohl                    
0000b805  lwip_ntohs                    
20017770  lwip_stats                    
00003511  main                          
00009575  mem_free                      
00009991  mem_init                      
00005829  mem_malloc                    
0000568d  mem_trim                      
0000b351  memcmp                        
00009171  memcpy                        
0000a441  memp_free                     
00006ac9  memp_init                     
00008b0d  memp_malloc                   
00009b0b  memset                        
0000978d  netif_add                     
20017a6c  netif_default                 
00008097  netif_init                    
20017a70  netif_list                    
0000b1d5  netif_set_addr                
0000b799  netif_set_default             
0000b073  netif_set_down                
0000b5a9  netif_set_gw                  
00007e59  netif_set_ipaddr              
0000b375  netif_set_link_down           
0000a495  netif_set_link_up             
0000b5c5  netif_set_netmask             
0000ac71  netif_set_up                  
000040a5  pbuf_alloc                    
0000a8dd  pbuf_cat                      
0000b747  pbuf_chain                    
0000b0a1  pbuf_clen                     
00006575  pbuf_copy                     
00007381  pbuf_copy_partial             
00008bb5  pbuf_free                     
20017a96  pbuf_free_ooseq_pending       
00007635  pbuf_header                   
000082cd  pbuf_realloc                  
0000b397  pbuf_ref                      
20000000  ram_heap                      
00008439  raw_input                     
00008e53  stats_init                    
0000b7ad  strlen                        
0000b815  sys_arch_protect              
0000b5e1  sys_arch_unprotect            
0000b881  sys_now                       
000079a1  sys_timeout                   
0000a681  sys_timeouts_init             
00008155  tcp_abandon                   
0000b841  tcp_abort                     
20017a74  tcp_active_pcbs               
20017a97  tcp_active_pcbs_changed       
0000644d  tcp_alloc                     
0000bc50  tcp_backoff                   
00007711  tcp_bind                      
20017a78  tcp_bound_pcbs                
0000b47d  tcp_close                     
000054e5  tcp_connect                   
0000aa79  tcp_eff_send_mss              
000059b1  tcp_enqueue_flags             
000095fd  tcp_fasttmr                   
0000945b  tcp_init                      
000013d1  tcp_input                     
20017a7c  tcp_input_pcb                 
0000a28d  tcp_keepalive                 
20017a80  tcp_listen_pcbs               
0000b897  tcp_new                       
0000b5fd  tcp_next_iss                  
000039fd  tcp_output                    
0000bc40  tcp_pcb_lists                 
00009ea1  tcp_pcb_purge                 
00008f95  tcp_pcb_remove                
0000bc80  tcp_persist_backoff           
00008211  tcp_process_refused_data      
0000ad21  tcp_recv_null                 
0000a895  tcp_recved                    
00009a0d  tcp_rexmit                    
000093cd  tcp_rexmit_fast               
0000a6d1  tcp_rexmit_rto                
0000920d  tcp_rst                       
0000b1ff  tcp_seg_copy                  
0000b49d  tcp_seg_free                  
0000b4bd  tcp_segs_free                 
0000a045  tcp_send_empty_ack            
0000a1d7  tcp_send_fin                  
0000b7c1  tcp_sent                      
00001de5  tcp_slowtmr                   
20017a84  tcp_ticks                     
0000ae75  tcp_timer_needed              
20017a88  tcp_tmp_pcb                   
0000b4dd  tcp_tmr                       
20017a8c  tcp_tw_pcbs                   
00009bf5  tcp_update_rcv_ann_wnd        
00001951  tcp_write                     
000078c9  tcp_zero_window_probe         
0000aabd  tivaif_init                   
0000a2e5  tivaif_interrupt              
00009035  tivaif_process_phy_interrupt  
00007f19  udp_bind                      
000094e9  udp_connect                   
00009c6b  udp_init                      
00002d61  udp_input                     
0000b3b9  udp_new                       
20017a90  udp_pcbs                      
0000b633  udp_recv                      
0000a33d  udp_remove                    
00006691  udp_sendto_if                 
0000afb5  usprintf                      
0000a395  ustrncpy                      
0000222d  uvsnprintf                    


GLOBAL SYMBOLS: SORTED BY Symbol Address 

address   name                          
-------   ----                          
00000000  __TI_static_base__            
00000000  g_pfnVectors                  
00000800  __STACK_SIZE                  
000013d1  tcp_input                     
00001951  tcp_write                     
00001de5  tcp_slowtmr                   
0000222d  uvsnprintf                    
00002a55  UARTvprintf                   
00002d61  udp_input                     
00002ff9  ip_input                      
00003511  main                          
00003791  PinoutSet                     
000039fd  tcp_output                    
000040a5  pbuf_alloc                    
000042b3  ipaddr_aton                   
000044b9  SysCtlClockFreqSet            
000048b5  icmp_input                    
00004a99  etharp_query                  
00004fd5  __aeabi_dsub                  
00004fdf  __aeabi_dadd                  
0000518d  InitDMADescriptors            
0000533d  etharp_output                 
000054e5  tcp_connect                   
0000568d  mem_trim                      
00005829  mem_malloc                    
000059b1  tcp_enqueue_flags             
00005c99  GPIOPadConfigSet              
00005e05  autoip_tmr                    
000061e9  __aeabi_ddiv                  
0000644d  tcp_alloc                     
00006575  pbuf_copy                     
00006691  udp_sendto_if                 
000069c5  etharp_raw                    
00006ac9  memp_init                     
00006cd1  dhcp_start                    
00006ec9  __aeabi_dmul                  
00006fc5  ethernet_input                
000070bd  lwIPInit                      
000071ad  ip_output_if                  
00007299  dhcp_release                  
00007381  pbuf_copy_partial             
00007635  pbuf_header                   
00007711  tcp_bind                      
000078c9  tcp_zero_window_probe         
000079a1  sys_timeout                   
00007b45  echoClientInit                
00007c11  TcpSendPacket                 
00007cd5  connectCallback               
00007d99  etharp_tmr                    
00007e59  netif_set_ipaddr              
00007f19  udp_bind                      
00008097  netif_init                    
00008155  tcp_abandon                   
00008211  tcp_process_refused_data      
000082cd  pbuf_realloc                  
00008383  __aeabi_idiv0                 
00008383  __aeabi_ldiv0                 
00008439  raw_input                     
000085a1  dhcp_renew                    
000087b5  autoip_arp_reply              
00008b0d  memp_malloc                   
00008bb5  pbuf_free                     
00008e53  stats_init                    
00008ef5  inet_chksum_pbuf              
00008f95  tcp_pcb_remove                
00009035  tivaif_process_phy_interrupt  
000090d5  lwIPHostTimerHandler          
00009171  __aeabi_memcpy                
00009171  __aeabi_memcpy4               
00009171  __aeabi_memcpy8               
00009171  memcpy                        
0000920d  tcp_rst                       
000092a5  autoip_start                  
000093cd  tcp_rexmit_fast               
0000945b  tcp_init                      
0000945d  lwIPEthernetIntHandler        
000094e9  udp_connect                   
00009575  mem_free                      
000095fd  tcp_fasttmr                   
00009685  ip_route                      
0000978d  netif_add                     
00009991  mem_init                      
00009a0d  tcp_rexmit                    
00009a89  ADCSequenceStepConfigure      
00009b03  __aeabi_memclr                
00009b03  __aeabi_memclr4               
00009b03  __aeabi_memclr8               
00009b05  __aeabi_memset                
00009b05  __aeabi_memset4               
00009b05  __aeabi_memset8               
00009b0b  memset                        
00009b7d  EMACInit                      
00009bf5  tcp_update_rcv_ann_wnd        
00009c6b  udp_init                      
00009c6d  UARTStdioConfig               
00009dc7  ip4_addr_isbroadcast          
00009ea1  tcp_pcb_purge                 
00009f0d  IntEnable                     
00009f75  __TI_decompress_lzss          
0000a045  tcp_send_empty_ack            
0000a0ad  UARTwrite                     
0000a111  etharp_cleanup_netif          
0000a175  dhcp_network_changed          
0000a1d7  tcp_send_fin                  
0000a235  EMACPHYConfigSet              
0000a28d  tcp_keepalive                 
0000a2e5  tivaif_interrupt              
0000a33d  udp_remove                    
0000a395  ustrncpy                      
0000a3ed  dhcp_fine_tmr                 
0000a441  memp_free                     
0000a495  netif_set_link_up             
0000a58f  dhcp_stop                     
0000a5e1  SysCtlPeripheralReset         
0000a631  dhcp_coarse_tmr               
0000a681  sys_timeouts_init             
0000a6d1  tcp_rexmit_rto                
0000a721  ADCSequenceConfigure          
0000a771  ip_output                     
0000a895  tcp_recved                    
0000a8dd  pbuf_cat                      
0000a925  DisplayIPAddress              
0000a969  __TI_auto_init_nobinit_nopinit
0000aa35  __aeabi_d2uiz                 
0000aa79  tcp_eff_send_mss              
0000aabd  tivaif_init                   
0000ab01  __aeabi_uidiv                 
0000ab01  __aeabi_uidivmod              
0000ab81  adcConfigure                  
0000ac71  netif_set_up                  
0000acad  EMACIntEnable                 
0000ad21  tcp_recv_null                 
0000ad5d  EMACConfigSet                 
0000ad95  SysCtlPeripheralReady         
0000ae3d  etharp_request                
0000ae75  tcp_timer_needed              
0000aee5  EMACConfigGet                 
0000af19  EMACIntClear                  
0000af4d  SysCtlPeripheralEnable        
0000af81  _c_int00_noargs               
0000afb5  usprintf                      
0000afe7  dhcp_arp_reply                
0000b017  ADCIntStatus                  
0000b073  netif_set_down                
0000b0a1  pbuf_clen                     
0000b0cf  EMACIntStatus                 
0000b0fb  GPIODirModeSet                
0000b129  SysTickIntHandler             
0000b155  lwip_htonl                    
0000b1d5  netif_set_addr                
0000b1ff  tcp_seg_copy                  
0000b229  lwIPTimer                     
0000b251  EMACPHYRead                   
0000b277  EMACPHYWrite                  
0000b29d  IntPrioritySet                
0000b2c1  UARTprintf                    
0000b32d  lwip_htons                    
0000b351  memcmp                        
0000b375  netif_set_link_down           
0000b397  pbuf_ref                      
0000b3b9  udp_new                       
0000b3fd  autoip_network_changed        
0000b41d  lwip_init                     
0000b45d  __aeabi_ui2d                  
0000b47d  tcp_close                     
0000b49d  tcp_seg_free                  
0000b4bd  tcp_segs_free                 
0000b4dd  tcp_tmr                       
0000b4fd  ADCSequenceDataGet            
0000b51b  EMACAddrGet                   
0000b58d  lwIPLocalIPAddrGet            
0000b5a9  netif_set_gw                  
0000b5c5  netif_set_netmask             
0000b5e1  sys_arch_unprotect            
0000b5fd  tcp_next_iss                  
0000b619  GPIOPinTypeGPIOOutput         
0000b633  udp_recv                      
0000b64d  ADCProcessorTrigger           
0000b67d  inet_chksum                   
0000b695  ipaddr_addr                   
0000b6ad  EMACReset                     
0000b6c3  EMACRxEnable                  
0000b6d9  EMACTxEnable                  
0000b6ef  GPIOPinTypeEthernetLED        
0000b71b  autoip_stop                   
0000b731  icmp_dest_unreach             
0000b747  pbuf_chain                    
0000b75d  FlashUserGet                  
0000b771  SysTickEnable                 
0000b785  SysTickIntEnable              
0000b799  netif_set_default             
0000b7ad  strlen                        
0000b7c1  tcp_sent                      
0000b7d5  EMACFrameFilterSet            
0000b7e5  IntMasterEnable               
0000b7f5  SysTickPeriodSet              
0000b805  lwip_ntohs                    
0000b815  sys_arch_protect              
0000b825  ADCSequenceEnable             
0000b833  __TI_decompress_none          
0000b841  tcp_abort                     
0000b84f  CPUcpsie                      
0000b85d  SysCtlMOSCConfigSet           
0000b869  __TI_zero_init                
0000b875  lwip_ntohl                    
0000b881  sys_now                       
0000b88d  ADCIntClear                   
0000b897  tcp_new                       
0000b8a1  EMACPowerManagementStatusGet  
0000b8a9  EMACTxDMAPollDemand           
0000b8b1  EMACRxDMADescriptorListSet    
0000b8b7  EMACTimestampIntStatus        
0000b8bd  EMACTxDMADescriptorListSet    
0000b8c3  GPIOPinRead                   
0000b8c9  GPIOPinWrite                  
0000b8cf  ResetISR                      
0000b8d5  SysCtlDelay                   
0000b8db  _system_pre_init              
0000b8df  C$$EXIT                       
0000b8df  abort                         
0000bc40  tcp_pcb_lists                 
0000bc50  tcp_backoff                   
0000bc80  tcp_persist_backoff           
0000bc87  ethbroadcast                  
0000bc8d  ethzero                       
0000bc94  ip_addr_any                   
0000bc98  ip_addr_broadcast             
0000bcdc  __TI_Handler_Table_Base       
0000bce8  __TI_Handler_Table_Limit      
0000bcf0  __TI_CINIT_Base               
0000bd00  __TI_CINIT_Limit              
20000000  __start___llvm_prf_cnts       
20000000  __stop___llvm_prf_cnts        
20000000  ram_heap                      
200172f0  g_pTxDescriptors              
20017650  g_pRxDescriptors              
20017770  lwip_stats                    
200179e0  dhcp_rx_options_val           
20017a38  dhcp_rx_options_given         
20017a48  current_header                
20017a4c  current_iphdr_dest            
20017a50  current_iphdr_src             
20017a54  current_netif                 
20017a58  g_pfnTimerHandler             
20017a5c  g_ui32AbnormalInts            
20017a60  g_ui32IPAddress               
20017a64  g_ui32NormalInts              
20017a68  g_ui32SysClock                
20017a6c  netif_default                 
20017a70  netif_list                    
20017a74  tcp_active_pcbs               
20017a78  tcp_bound_pcbs                
20017a7c  tcp_input_pcb                 
20017a80  tcp_listen_pcbs               
20017a84  tcp_ticks                     
20017a88  tcp_tmp_pcb                   
20017a8c  tcp_tw_pcbs                   
20017a90  udp_pcbs                      
20017a94  err                           
20017a95  g_bLED                        
20017a96  pbuf_free_ooseq_pending       
20017a97  tcp_active_pcbs_changed       
20017a98  __stack                       
20018298  __STACK_END                   
20018298  __STACK_TOP                   
2001829c  g_ui32LocalTimer              
200182d0  g_RxDescList                  
200182e0  g_TxDescList                  
200182f0  g_ui32tcpPollTick             
200182f4  g_bIPAddrValid                
200182f5  g_bconnect                    
200182f8  g_ui32sysTick                 
ffffffff  __TI_pprof_out_hndl           
ffffffff  __TI_prof_data_size           
ffffffff  __TI_prof_data_start          
ffffffff  __binit__                     
ffffffff  __c_args__                    
ffffffff  binit                         
UNDEFED   __mpu_init                    
UNDEFED   _system_post_cinit            

[280 symbols]
